S00C0000546573742E7372656378
S11300000C943A000C9444000C9444000C94440066
S11300100C9444000C9444000C9444000C9444004C
S11300200C9444000C9444000C9444000C9444003C
S11300300C9444000C9444000C9444000C9444002C
S11300400C9444000C9444000C9444000C9444001C
S11300500C9444000C9444000C9444000C9444000C
S11300600C9444000C9444000C9444000C944400FC
S11300700C94440011241FBECFEFD4E0DEBFCDBFEB
S11300800E9446000C944E000C94000084B1806ED3
S113009084B990E485B1892785B9FCCFF894FFCF62
S9030000FC
